:100000001DC037C036C035C034C033C032C031C067
:1000100030C02FC02EC02EC0B9C02BC02AC029C0EE
:1000200028C027C026C031C53BC545C56EC576C5AD
:1000300079C57CC57FC582C595C597C511241FBEEE
:10004000CFE5D4E0DEBFCDBF10E0A0E6B0E0ECEF3E
:10005000FEE102C005900D92A836B107D9F711E074
:10006000A8E6B0E001C01D92AA30B107E1F75CD864
:1000700043CFC6CF1F920F920FB60F9211242F932A
:100080003F934F935F936F938F939F93EF93FF9360
:100090008BB16CB188718093DA004091DB00509194
:1000A000DC004F5F5F4F4F7150708091DD00909189
:1000B000DE004817590721F482E08093DA004FC030
:1000C0002091060130910701809104019091050172
:1000D00028173907BCF58091040190910501892BFF
:1000E00089F18091060190910701FC01EF51FF4FCA
:1000F000208101969093070180930601332727FD05
:100100003095862F90E028173907E1F0559892989E
:1001100010926A00109205011092040110920301DE
:100120001092020110920701109206018091DF00E7
:100130009091E00001969093E0008093DF0080E1D1
:10014000809301015093DC004093DB00E091DB00E1
:10015000F091DC00E654FF4F60836A3049F48091EF
:10016000DF009091E00001969093E0008093DF0023
:10017000FF91EF919F918F916F915F914F913F917F
:100180002F910F900FBE0F901F9018951F920F92F6
:100190000FB60F9211242F933F938F939F93EF935A
:1001A000FF9320910201309103018091040190910D
:1001B00005012817390734F4809102019091030159
:1001C000809734F0559880910401909105010AC000
:1001D0008091020190910301FC01EF51FF4F2081BA
:1001E0002CB901969093030180930201FF91EF9146
:1001F0009F918F913F912F910F900FBE0F901F9065
:1002000018951092DA001092DC001092DB00109228
:10021000DE001092DD001092E0001092DF001092DC
:100220000101109203011092020110920501109237
:100230000401109207011092060110920901109218
:10024000080110BC8FE289B988E98AB986E880BDC7
:1002500080E090E02EE2FC01EF51FF4F20830196F9
:1002600080329105C1F708952091DB003091DC00C8
:100270008091DD009091DE0040E050E028173907C2
:1002800011F441E050E0CA0108952091020130913B
:100290000301809104019091050140E050E028178E
:1002A000390711F441E050E0CA0108952091DF00C0
:1002B0003091E0008091DF009091E000892B49F0BF
:1002C0008091DF009091E00001979093E00080938F
:1002D000DF00C9010895559810920501109204019C
:1002E0001092030110920201109207011092060170
:1002F000109209011092080108952091DD003091BB
:10030000DE008091DB009091DC002817390759F45A
:100310001092DE001092DD001092DC001092DB00E3
:1003200040E051E01BC08091DD009091DE0001961D
:100330008F7190709093DE008093DD00E091DD007E
:10034000F091DE00E654FF4F20818091DA0099277A
:1003500087FD9095582F4427420F511DCA010895DB
:10036000482F209102013091030180910401909166
:10037000050128173907A9F7559880910801909130
:10038000090180976CF48091080190910901FC01AA
:10039000EF51FF4F4083019690930901809308012C
:1003A00008958F708A3018F0482F495C02C0482F9A
:1003B000405D2091020130910301809104019091F0
:1003C000050128173907A9F75598809108019091E0
:1003D000090180976CF48091080190910901FC015A
:1003E000EF51FF4F408301969093090180930801DC
:1003F00008951F93182F82958F70D3DF812FD1DF3F
:100400001F91089520910201309103018091040110
:100410009091050128173907A9F755981092030103
:1004200010920201809108019091090190930501B9
:1004300080930401109207011092060110920901A5
:1004400010920801559A0895AF92BF92CF92DF9211
:10045000EF92FF920F931F93CF93DF935B016C0199
:10046000B5D7EB01C601B50126E636E646EE54E403
:1004700071D97B018C0120E030E040E85FE3B5DA20
:1004800088231CF461E070E020C0C801B70120E0BF
:100490003FEF4FE757E453DA1816A4F4C601B5014D
:1004A00020E030E040E251E455D990D788EB90E06D
:1004B00005C0FC013197F1F761507040611571057D
:1004C000C1F706C0C801B70181D7CB010197F1F789
:1004D00080918600909187008C0F9D1F90938700DC
:1004E0008093860080918800909189008C0F9D1FD9
:1004F000909389008093880080918A0090918B006E
:10050000C817D90758F480918A0090918B008C1BF2
:100510009D0B90938B0080938A0013C080918A007A
:1005200090918B00892B69F08091DF009091E00021
:1005300001969093E0008093DF0010928B00109260
:100540008A00DF91CF911F910F91FF90EF90DF9084
:10055000CF90BF90AF90089522B3277080FF02C064
:10056000C09A01C0C09881FD206882FD206483FD8F
:10057000206284FD206185FD286022BB08951F93C1
:10058000182F81E080936A00929A60E070E080E02A
:1005900090E45ADF559810920501109204011092D0
:1005A00003011092020110920701109206011092AD
:1005B00009011092080120910201309103018091FC
:1005C00004019091050128173907B9F0929810920B
:1005D0006A005598109205011092040110920301CF
:1005E0001092020110920701109206011092090167
:1005F0001092080121E030E064C0209102013091A6
:100600000301809104019091050128173907A9F78A
:1006100055988091080190910901809774F4809118
:10062000080190910901FC01EF51FF4F2AE020835E
:100630000196909309018093080120910201309165
:100640000301809104019091050128173907A9F74A
:1006500055988091080190910901809774F48091D8
:10066000080190910901FC01EF51FF4F2AE220831C
:100670000196909309018093080120910201309125
:100680000301809104019091050128173907A9F70A
:100690005598809108019091090180976CF48091A0
:1006A000080190910901FC01EF51FF4F1083019661
:1006B000909309018093080180917D009ADE20E0EB
:1006C00030E0C9011F91089585E459DF892B09F0B5
:1006D00046C080917E008DDE2091020130910301A1
:1006E000809104019091050128173907A9F75598C1
:1006F0008091080190910901809774F4809108011C
:1007000090910901FC01EF51FF4F2AE020830196EF
:10071000909309018093080110927E0020910201BC
:100720003091030180910401909105012817390748
:10073000A9F75598109203011092020180910801C7
:100740009091090190930501809304011092070193
:10075000109206011092090110920801559A08950D
:1007600083E50DDF892B09F056C08091820041DEC0
:10077000809183003EDE209102013091030180913F
:1007800004019091050128173907A9F75598809120
:10079000080190910901809774F48091080190916B
:1007A0000901FC01EF51FF4F2AE02083019690934D
:1007B00009018093080180918E008F5F80938E00E5
:1007C00080918E00893018F081E080938E0081E066
:1007D00080938D00209102013091030180910401EA
:1007E0009091050128173907A9F755981092030130
:1007F00010920201809108019091090190930501E6
:1008000080930401109207011092060110920901D1
:1008100010920801559A0895EF92FF920F931F933B
:10082000082F8FE4ACDE892B09F05CC0802FE1DD5E
:1008300010E0000F111F000F111F50E9E52E50E0CE
:10084000F52EE00EF11EF7018081D3DDF7018181E5
:10085000D0DD0E561F4FF8018081CBDDF70183817B
:10086000C8DD209102013091030180910401909133
:10087000050128173907A9F755988091080190912B
:100880000901809774F48091080190910901FC019D
:10089000EF51FF4F2AE02083019690930901809346
:1008A000080120910201309103018091040190918F
:1008B000050128173907A9F75598109203011092DE
:1008C00002018091080190910901909305018093A4
:1008D0000401109207011092060110920901109272
:1008E0000801559A1F910F91FF90EF900895982F4E
:1008F0008D3338F08AE0989F900111242C513240BA
:1009000002C0282F30E0C9010895AF92BF92CF9264
:10091000DF92EF92FF920F931F93CF93DF93D82E26
:10092000C62EB42E8091860090918700845F9140FE
:10093000A8F08091860090918700845F9140909309
:100940008700809386008091800082FF07C080919D
:100950007D008F3F19F081E080938C0080918800AA
:1009600090918900885E934010F4EE240CC0809131
:10097000880090918900885E9340909389008093CD
:100980008800EE24E39440E050E0C1E0D0E07AE05B
:10099000F72EAA24A394CE01042E02C0880F991F1B
:1009A0000A94E2F7282FEE20C9F0FA01EE0FFF1F9C
:1009B000E255FF4F80819181892B81F08081918167
:1009C00001979183808380819181892B39F4909163
:1009D0008300822F8095892380938300FA01EE0F94
:1009E000FF1FEE0FFF1FE057FF4F80818D1509F0AD
:1009F000E8C08181BE0102C0660F771F8A95E2F7C9
:100A0000FA01EE0FFF1FEE0FFF1FEE56FF4F108192
:100A10000C2D0623A02FB0E0FA01E855FF4F80818E
:100A2000992787FD9095A817B90719F480E090E001
:100A300006C0808190E0811191E09A25892F782F5E
:100A4000FA01E855FF4F8081992787FD9095A817F7
:100A5000B90719F480E090E007C0808190E0882316
:100A600009F491E09A25892F382F812F90E0A0E09A
:100A7000B0E08F709070A070B070FC018B30910569
:100A800008F09BC0ED5EFF4F099490918300822F88
:100A90008095892380938300002309F48EC031C0A0
:100AA00090918300822F80958923809383006B210E
:100AB00009F483C026C0FA01EE0FFF1FEE0FFF1FDF
:100AC000E057FF4F8381863008F077C08381BE01F5
:100AD00002C0660F771F8A95E2F7362F9091830048
:100AE000822F8095892380938300002329F08091B1
:100AF0008200382331F061C080918200382309F4EC
:100B00005CC080918300282B06C0772309F455C070
:100B1000809183002827209383004FC0332309F45A
:100B20004CC0F6CF772309F448C02AC0332309F418
:100B300044C026C0772309F440C002C03323E9F142
:100B4000FA01EE0FFF1FE255FF4F80819181892B43
:100B5000B9F080918300209528232093830011828F
:100B600010822BC0772349F102C0332331F1FA01FF
:100B7000EE0FFF1FE255FF4F80819181892BE9F431
:100B800080918300282B20938300FA01EE0FFF1F32
:100B9000EE0FFF1FE057FF4F83818D3330F08F9DA5
:100BA000C00111248C51924001C090E0FA01EE0F77
:100BB000FF1FE255FF4F91838083FA01E855FF4FF5
:100BC00000834F5F5F4F4630510509F0E4CEDF915F
:100BD000CF911F910F91FF90EF90DF90CF90BF903A
:100BE000AF90089583B38F738093690086B38C713F
:100BF000809368008091680090917F009827809191
:100C0000680080937F0020918000892F8095822347
:100C10008093800080916800982390936800909161
:100C2000800080916800892B80938000809169000A
:100C30009091810098278091690080938100209194
:100C40008200892F809582238093820080916900A1
:100C50009823909369009091820080916900892B7C
:100C60008093820008951F9310928B0010928A0047
:100C700088B392E0892788BB2091DD003091DE00A7
:100C80008091DB009091DC002817390759F410920D
:100C9000DE001092DD001092DC001092DB0040E0DC
:100CA00051E01BC08091DD009091DE0001968F71B4
:100CB00090709093DE008093DD00E091DD00F09174
:100CC000DE00E654FF4F20818091DA00992787FDEE
:100CD0009095582F4427420F511D10926B00A0E0B1
:100CE000B0E060E070E010E087C0CA018070892B3E
:100CF00009F087C0842F109719F440936B003FC010
:100D0000A130B10519F440936C0039C0A0FF1EC09A
:100D1000403398F04A3318F4942F90530FC0413465
:100D200060F0473418F4942F975308C0413628F0E8
:100D3000473618F4942F975501C090E0192BFB010A
:100D4000E359FF4F10836F5F7F4F19C0403398F016
:100D50004A3318F4942F90530FC0413460F0473455
:100D600018F4942F975308C0413628F0473618F4EA
:100D7000942F975501C090E0192F1295107F8A305B
:100D800009F43FC080916B008A3221F080916B00A2
:100D9000833209F411962091DD003091DE008091BC
:100DA000DB009091DC002817390759F41092DE001F
:100DB0001092DD001092DC001092DB0040E051E068
:100DC0001BC08091DD009091DE0001968F719070C4
:100DD0009093DE008093DD00E091DD00F091DE0075
:100DE000E654FF4F20818091DA00992787FD909586
:100DF000582F4427420F511D81E04030580709F019
:100E000074CF80916B008A3209F0E4C063307105C1
:100E100091F480916C00833591F490916D008091F4
:100E20007D00981761F080916D0060916E00409197
:100E30006F006BDDCFC06115710509F4CBC09091D7
:100E40006D0080917D00981709F0C4C080916C00FE
:100E50008C3409F458C08D3438F4843409F498C0C3
:100E6000873409F0B2C040C0813509F442C08335EF
:100E700009F0ABC06330710509F0A7C08091010192
:100E8000882309F0A2C09091840080918200981775
:100E900049F49091850080918300981719F410927D
:100EA0008C0003C081E080938C0080916E00809361
:100EB000840080916F008093850010928E00909145
:100EC000840080918200981709F07FC0909185007E
:100ED00080918300981709F078C010928D001092CD
:100EE00087001092860071C06130710509F06AC0F8
:100EF00065C080916E00863008F064C06230710574
:100F000009F060C040C080916E00863008F05AC081
:100F10006630710509F056C0E0916E00F0E08091F6
:100F20006F00EE0FFF1FEE0FFF1FE057FF4F808394
:100F3000E0916E00F0E080917000EE0FFF1FEE0F69
:100F4000FF1FE057FF4F8183E0916E00F0E080913A
:100F50007100EE0FFF1FEE0FFF1FEE56FF4F808355
:100F6000E0916E00F0E080917200EE0FFF1FEE0F37
:100F7000FF1FE057FF4F838380E990E061E070E05E
:100F800048E150E0A3D780916E0080938F001DC090
:100F900062307105B9F490916E0080917D009817D0
:100FA00069F08091800082FF09C080916E0080937B
:100FB0007D0060917D0080E090E091D781E080939A
:100FC0008C0003C081E080937E0060E070E080E8E8
:100FD00090E43ADA1F910895EF92FF920F931F93D6
:100FE000CF93DF9310917D00FDDD60E070E080E243
:100FF00091E42ADAF7DD80918000887111F000E039
:1010000012C0C19860E070E080E89FE31DDAEADD7D
:101010008091800088718831A9F7103418F001E0C0
:101020001FE301C001E0F0908000C0E0D0E052E09A
:10103000E52E69C060E070E080E291E405DAD2DD7F
:101040002196CA31D1056CF080917D0090E08F73BC
:101050009070212F30E08217930709F40E25C0E02D
:10106000D0E080917D0090E08F739070212F30E070
:101070008217930709F00D7F01FF03C010928300D0
:1010800004C0812F8F73809383008091830064DA82
:10109000809180002F2D30E090E08227932783FFFE
:1010A00002C0F3FE11508091800090E082279327C8
:1010B00084FF02C024FF1F5FF0908000112311F411
:1010C0001FE303C0103408F011E0809180008871A4
:1010D00039F019C060E070E080E89FE3B5D982DDA7
:1010E0008091800088718831A9F71F3309F41FEFC0
:1010F00080917D00181751F080E090E0612FEFD6CD
:1011000010937D0003C0002309F094CF1092830058
:1011100010927E00809183001FDADF91CF911F91A2
:101120000F91FF90EF900895AF92BF92CF92DF9210
:10113000EF92FF920F931F93CF93DF9383E087BBD0
:1011400014BA8CEF81BB8EE188BB15BA12BA10922B
:1011500068001092800010927F0010926900109237
:1011600082001092810010926A00109283008FEF2B
:1011700080938400809385001092870010928600EF
:10118000109289001092880010928B0010928A00B1
:1011900010928C0010928D0080938F00E199FECF09
:1011A00080E090E08BD680937D0080E990E061E064
:1011B00070E048E150E072D624D878940DDFC19AEF
:1011C00092980091800010E0BB24B39474E1C72E84
:1011D000D12CAA24AA9461E0E62EF12C03DD8091A3
:1011E0007D0060918200409183008FDB80918000C0
:1011F000202F30E090E08227932784FF0BC004FD6E
:1012000009C003FF03C0B0928C0004C01F5F1830F8
:1012100008F011E08091800090E08227932783FFFF
:1012200006C023FF04C0112311F424FD17E08091B0
:10123000800090E08227932783FF02C023FF10E005
:10124000009180002091DB003091DC008091DD0076
:101250009091DE002817390761F080918A00909103
:101260008B00892B31F4D0928B00C0928A0001C090
:10127000FADC2091DF003091E0008091DF00909156
:10128000E000892B49F08091DF009091E000019708
:101290009093E0008093DF00232B51F72091DB0037
:1012A0003091DC008091DD009091DE002817390735
:1012B00021F580917E00882311F006DA1EC080910E
:1012C0008F008F3F31F080918F00A6DAA0928F00BF
:1012D00014C09091840080918200981769F49091D5
:1012E000850080918300981739F480918C008823C1
:1012F00019F480918D00811133DA809101018823E6
:1013000041F01092010180918E00882311F4B09277
:101310008E0020910201309103018091040190918F
:1013200005012817390761F480916A00882341F08C
:1013300060E070E080E090E487D8929810926A00B4
:10134000112379F0173011F48FE30DC0812F90E055
:101350000197970102C0220F331F8A95E2F7C90156
:1013600002C080918300F8D880918E00882341F1DB
:1013700060E070E080E090E467D8C0E0D0E006C0B4
:1013800060E070E080E090E45FD8219680918E006C
:1013900090E0C817D907A4F380918E0020917D00BA
:1013A00090E00197A70102C0440F551F8A95E2F70C
:1013B000242309F413CF60E070E080E090E404C0DF
:1013C00060E070E080E89FE33FD808CFEF92FF92A3
:1013D0000F931F937B018C0120E030E040E05FE43D
:1013E000D9D288237CF0C801B70120E030E040E08A
:1013F0005FE45ED125D39B01AC01205030404040DA
:10140000504805C0C801B7011BD39B01AC01B9010D
:10141000CA011F910F91FF90EF900895A0E0B0E0F6
:10142000E3E1FAE004C5DC012B01FA019C91923062
:1014300008F439C1EB018881823008F433C194305B
:1014400069F4843009F02FC111969C91119789811C
:10145000981709F428C1A0E6B0E025C1843009F44A
:1014600021C18230A9F4923009F01DC19A01AD0169
:1014700088E0EA010990AE01E90109929E018150DC
:10148000C1F7E201898111969C918923818308C16A
:10149000923009F407C112962D903C901397EB01FE
:1014A0008A819B811496AD90BD90CD90DC9017976A
:1014B000EC80FD800E811F819101281B390BB90141
:1014C00037FF04C066277727621B730B60327105F4
:1014D0000CF061C0121613066CF537014801062E98
:1014E00004C096948794779467940A94D2F721E085
:1014F00030E040E050E004C0220F331F441F551F6E
:101500006A95D2F721503040404050402E213F2173
:1015100040235123211531054105510521F021E0DA
:1015200030E040E050E079018A01E628F7280829F8
:1015300019293CC0232BD1F1260E371E3501460157
:10154000062E04C096948794779467940A94D2F7F1
:1015500021E030E040E050E004C0220F331F441F80
:10156000551F6A95D2F721503040404050402A2103
:101570003B214C215D21211531054105510521F00B
:1015800021E030E040E050E059016A01A628B72888
:10159000C828D9280BC0821593052CF01C01AA2459
:1015A000BB24650103C0EE24FF24870111969C91A2
:1015B000D20111968C91981709F445C0992339F0FE
:1015C000A80197012A193B094C095D0906C0A6012B
:1015D00095012E193F09400B510B57FD08C0118290
:1015E0003382228224833583468357831DC081E062
:1015F00081833382228288279927DC01821B930B07
:10160000A40BB50B84839583A683B7830DC0220FEB
:10161000331F441F551F248335834683578382819C
:1016200093810197938382832481358146815781F9
:10163000DA01C9010197A109B1098F5F9F4FAF4F2F
:10164000BF4328F30BC0918333822282EA0CFB1C38
:101650000C1D1D1DE482F5820683178383E08083C1
:10166000248135814681578157FF1AC0C901AA27B5
:1016700097FDA095BA2F81709070A070B0705695AC
:10168000479537952795822B932BA42BB52B8483D5
:101690009583A683B7838281938101969383828306
:1016A000DF0101C0D201CD01CDB7DEB7E2E1DBC37E
:1016B000A0E2B0E0EDE5FBE0C6C369837A838B83EB
:1016C0009C832D833E834F835887E9E0EE2EF12CD7
:1016D000EC0EFD1ECE010196B701D8D28E010F5E31
:1016E0001F4FCE010596B801D1D28A8991E0892792
:1016F0008A8BC701B801AE01475E5F4F8FDEF1D123
:10170000A096E6E0BCC3A0E2B0E0E8E8FBE09BC343
:1017100069837A838B839C832D833E834F83588791
:10172000F9E0EF2EF12CEC0EFD1ECE010196B70173
:10173000ADD28E010F5E1F4FCE010596B801A6D225
:10174000C701B801AE01475E5F4F68DECAD1A096FF
:10175000E6E095C3A0E2B0E0EFEAFBE068C369838E
:101760007A838B839C832D833E834F835887CE015E
:101770000196BE01675F7F4F89D2CE010596BE01FB
:101780006F5E7F4F83D29985923088F0898982304D
:10179000C8F0943019F4823051F404C0843029F434
:1017A000923081F480E690E0C6C0923049F420E0A7
:1017B0009A858A89981321E02A87CE010996BBC0B1
:1017C000823049F420E09A858A89981321E02A8B97
:1017D000CE014196B0C02D843E844F8458886D88D8
:1017E0007E888F88988CEE24FF248701AA24BB244E
:1017F000650140E050E060E070E0E0E0F0E0C10151
:1018000081709070892BE9F0E60CF71C081D191DFA
:101810009A01AB012A0D3B1D4C1D5D1D80E090E03F
:10182000A0E0B0E0E614F7040805190520F481E013
:1018300090E0A0E0B0E0BA01A901480F591F6A1F6B
:101840007B1FAA0CBB1CCC1CDD1C97FE08C081E0D2
:1018500090E0A0E0B0E0A82AB92ACA2ADB2A319693
:10186000E032F10549F0660C771C881C991C5694EF
:10187000479437942794C3CFFA85EA892B893C890A
:101880008B859C85280F391F2E5F3F4F17C0CA01DB
:1018900081709070892B61F016950795F794E79405
:1018A00080E090E0A0E0B0E8E82AF92A0A2B1B2BA0
:1018B00076956795579547952F5F3F4F77FDE7CF13
:1018C0000CC0440F551F661F771F17FD4160EE0CBB
:1018D000FF1C001F111F21503040403090E059077D
:1018E00090E0690790E4790760F32B8F3C8FDB0170
:1018F000CA018F779070A070B07080349105A105F7
:10190000B10561F447FD0AC0E114F10401051105B8
:1019100029F0405C5F4F6F4F7F4F40781A8EFE1763
:1019200011F081E08A8F4D8F5E8F6F8F78A383E0F7
:10193000898FCE014996D5D0A096E2E194C2A8E164
:10194000B0E0E4EAFCE07FC269837A838B839C8306
:101950002D833E834F83588789E0E82EF12CEC0ECF
:10196000FD1ECE010196B70191D18E010F5E1F4F72
:10197000CE010596B8018AD18985823038F08989EF
:10198000823020F0C701B801F9D101C08FEF68960D
:10199000E6E075C2A8E1B0E0EFECFCE054C2698378
:1019A0007A838B839C832D833E834F83588789E082
:1019B000E82EF12CEC0EFD1ECE010196B70166D18A
:1019C0008E010F5E1F4FCE010596B8015FD189854C
:1019D000823038F08989823020F0C701B801CED139
:1019E00001C08FEF6896E6E04AC2A8E1B0E0EAEFF6
:1019F000FCE029C269837A838B839C832D833E8399
:101A00004F83588789E0E82EF12CEC0EFD1ECE01A5
:101A10000196B7013BD18E010F5E1F4FCE01059697
:101A2000B80134D18985823038F08989823020F03C
:101A3000C701B801A3D101C081E06896E6E01FC2EA
:101A4000ACE0B0E0E5E2FDE002C269837A838B831B
:101A50009C83CE010196BE016B5F7F4F17D18D81B4
:101A6000823061F1823050F1843021F48E818823FC
:101A700051F12EC02F81388537FD20C06E812F3166
:101A800031051CF06623F9F023C08EE190E0821B43
:101A9000930B29853A854B855C8504C056954795FF
:101AA000379527958A95D2F76623B1F050954095E2
:101AB000309521953F4F4F4F5F4F0EC020E030E0F3
:101AC00040E050E009C02FEF3FEF4FEF5FE704C069
:101AD00020E030E040E050E8B901CA012C96E2E095
:101AE000D2C1DF92EF92FF920F931F93FC01E4802B
:101AF000F58006811781D1808081823048F480E0B2
:101B000090E0A0E1B0E0E82AF92A0A2B1B2BA5C03F
:101B1000843009F49FC0823021F4EE24FF24870131
:101B200005C0E114F1040105110519F4E0E0F0E04D
:101B300096C0628173819FEF623879070CF05BC0B9
:101B400022E83FEF261B370B2A3131052CF020E02D
:101B500030E040E050E02AC0B801A701022E04C0E6
:101B600076956795579547950A94D2F781E090E06E
:101B7000A0E0B0E004C0880F991FAA1FBB1F2A95E0
:101B8000D2F70197A109B1098E219F21A023B1238A
:101B90000097A105B10521F081E090E0A0E0B0E060
:101BA0009A01AB01282B392B4A2B5B2BDA01C90197
:101BB0008F779070A070B07080349105A105B10549
:101BC00039F427FF09C0205C3F4F4F4F5F4F04C0DF
:101BD000215C3F4F4F4F5F4FE0E0F0E02030A0E04E
:101BE0003A07A0E04A07A0E45A0710F0E1E0F0E06D
:101BF00079018A0127C06038710564F5FB01E1585D
:101C0000FF4FD801C7018F779070A070B0708034FB
:101C10009105A105B10539F4E7FE0DC080E490E01F
:101C2000A0E0B0E004C08FE390E0A0E0B0E0E80EF8
:101C3000F91E0A1F1B1F17FF05C016950795F7947D
:101C4000E794319687E016950795F794E7948A957F
:101C5000D1F705C0EE24FF248701EFEFF0E06E2FEF
:101C6000679566276795902F9F77D794DD24D79443
:101C70008E2F8695492F462B582F5D29B701CA0113
:101C80001F910F91FF90EF90DF900895FC01DB0111
:101C9000408151812281622F6F7770E0221F2227BD
:101CA000221F9381892F880F822B282F30E0991FC4
:101CB0009927991F11969C93119721153105A9F524
:101CC000411551056105710511F482E037C082E8C4
:101CD0009FEF13969C938E9312979A01AB0167E046
:101CE000220F331F441F551F6A95D1F783E08C9351
:101CF0000DC0220F331F441F551F12968D919C91CA
:101D00001397019713969C938E931297203080E03F
:101D1000380780E0480780E4580758F314962D935D
:101D20003D934D935C93179708952F3F310579F4B8
:101D3000411551056105710519F484E08C930895EE
:101D400064FF03C081E08C9312C01C9210C02F5717
:101D5000304013963C932E93129783E08C9387E048
:101D6000440F551F661F771F8A95D1F7706414962C
:101D70004D935D936D937C93179708951F93DC01AA
:101D8000FB019C91923008F447C08081823008F4B6
:101D900043C0943051F411961C91843099F581819F
:101DA000682F70E0611B71093FC0843021F09230D0
:101DB00031F48230B9F18181882389F12DC01196E7
:101DC0001C9111978230F1F081811817D9F4129685
:101DD0002D913C911397828193818217930794F000
:101DE00028173907BCF014968D919D910D90BC91E8
:101DF000A02D2481358146815781281739074A074C
:101E00005B0718F4112341F00AC082179307A40757
:101E1000B50740F4112319F061E070E005C06FEFE1
:101E20007FEF02C060E070E0CB011F9108952F9218
:101E30003F924F925F926F927F928F929F92AF925A
:101E4000BF92CF92DF92EF92FF920F931F93CF93A7
:101E5000DF93CDB7DEB7CA1BDB0B0FB6F894DEBF3E
:101E60000FBECDBF09942A88398848885F846E8464
:101E70007D848C849B84AA84B984C884DF80EE80AE
:101E8000FD800C811B81AA81B981CE0FD11D0FB6B7
:101E9000F894DEBF0FBECDBFED010895DC01CB018C
:101EA000FC01E199FECF06C0FFBBEEBBE09A319684
:101EB0000DB20D9241505040B8F70895E199FECF10
:101EC0009FBB8EBBE09A99278DB30895DC01CB01AF
:101ED00002C02D9105D041505040D8F70895262FCB
:101EE000E199FECF9FBB8EBB2DBB0FB6F894E29A53
:0C1EF000E19A0FBE01960895F894FFCF10
:00000001FF
